:020000040800F2
:10000000A8AB00209D010008090D0008090A00089E
:10001000050D0008FF0300081D1400080000000083
:10002000000000000000000000000000510F000868
:10003000F105000800000000190D0008B5010008D6
:10004000B7010008B7010008B7010008B7010008B0
:10005000B7010008B7010008B7010008B7010008A0
:10006000B7010008B7010008B7010008B701000890
:10007000B7010008B7010008B7010008B701000880
:10008000B7010008B7010008B7010008B701000870
:10009000B7010008B7010008B7010008B701000860
:1000A000B7010008B7010008B7010008B701000850
:1000B000B7010008B7010008B7010008B701000840
:1000C000B7010008B7010008B7010008B701000830
:1000D000B7010008B7010008B7010008B701000820
:1000E000B7010008B7010008B7010008B701000810
:1000F000B7010008B7010008B7010008B701000800
:10010000B7010008B7010008B7010008B7010008EF
:10011000B7010008B7010008B7010008B7010008DF
:10012000B7010008B7010008B7010008B7010008CF
:10013000B7010008B7010008B7010008B7010008BF
:10014000B7010008B7010008B7010008B7010008AF
:10015000B7010008B7010008B7010008B70100089F
:10016000B7010008B7010008B7010008B70100088F
:10017000B7010008B7010008B7010008B70100087F
:10018000B7010008B7010008DFF80CD000F096F8BE
:1001900000480047BD190008A8AB0020064880476A
:1001A00006480047FEE7FEE7FEE7FEE7FEE7FEE75C
:1001B000FEE7FEE7FEE7FEE7A5110008890100085B
:1001C00040EA01039B0703D009E008C9121F08C0D9
:1001D000042AFAD203E011F8013B00F8013B521E59
:1001E000F9D270470146002000E0401C0A5C002A5A
:1001F000FBD17047034611F8012B00F8012B002AB0
:10020000F9D11846704770B5064601F0F5F9046853
:1002100005460A220021304600F018F82C6070BD17
:1002200030B50B46014600202022012409E021FAC6
:1002300002F59D4205D303FA02F5491B04FA02F5C3
:100240002844151EA2F10102F1DC30BD2DE9F04772
:100250000F46914680460446002614F8015B2DB1F6
:1002600000F03EF80068405DC007F6D12B2D02D0AB
:100270002D2D18D0641E4A463946204600F034F829
:1002800027B13968A14201D1C7F8008071054FF04C
:1002900002040BD54042002803DD01F0ADF90460F3
:1002A000A007BDE8F08746F48066E4E70028F8DAA6
:1002B00001F0A2F904606FF00040F2E7064C074D30
:1002C00006E0E06840F0010394E807009847103426
:1002D000AC42F6D3FFF75CFFDC460008FC460008A2
:1002E00000487047D84600082DE9F05F8246007844
:1002F00000278B4615460AF10104B946302801D083
:100300009DB113E014F8010B0127782803D0582879
:1003100001D045B10AE00DB1102D07D100271025FD
:1003200014F8010B02E0082500E00A250026B0467B
:100330000EE005FB080005FB06F1012701EB104666
:100340001FFA80F8B6F5803F00D3B94614F8010BC8
:10035000294600F018F80028EBDABBF1000F05D0B1
:100360000FB1641E00E05446CBF80040B9F1000F15
:1003700006D001F041F902210160C81EBDE8F09FDE
:1003800048EA0640FAE73A2800D2303820F0200246
:10039000412A01D3A2F13700884201D34FF0FF3048
:1003A000704770B501EB020410F8015B15F007030C
:1003B00001D110F8013B2A1106D110F8012B03E0FE
:1003C00010F8016B01F8016B5B1EF9D12B0705D406
:1003D0000023521E0FD401F8013BFAE710F8013B4D
:1003E00002F10202A1EB030303E013F8015B01F841
:1003F000015B521EF9D5A142D6D3002070BD00BFCB
:10040000FEE70146302905DB392903DCA1F1300084
:10041000C0B27047612905DB662903DCA1F15700F2
:10042000C0B2F6E7412905DB462903DCA1F137001C
:10043000C0B2EEE73720ECE710B5484800684849FD
:10044000884208D24548001D46490860001F0068E0
:10045000454908601AE00A204449087000204870A5
:1004600088700F20C870FF200872FF213F4841723A
:1004700000218172C1720A203C49087100213B4869
:10048000417181710121C171002010BD38A000F0BF
:1004900061FD98B13948006800785B2804D137487D
:1004A0000068401C35490860002404E000F090FA20
:1004B0002E490855641C042CF8DB07E00A202B4960
:1004C00008700020487088700F20C8702CA000F0C1
:1004D00041FDA8B12948006800785B2804D127486D
:1004E0000068401C25490860002406E000F070FA0E
:1004F000C1B21E4808300155641C042CF6DB08E02C
:10050000FF201A490872FF211848417281720021A8
:10051000C1721EA000F01EFDA8B118480068007846
:100520005B2804D115480068401C14490860002469
:1005300006E000F04DFAC1B20C48001D0155641CE4
:10054000042CF6DB08E00A2008490871002107485E
:10055000417181710121C171002096E700000E08F0
:10056000C0D40100680000205C000020F0010020E1
:10057000435F49505F414444520000008400002022
:10058000435F49505F4D41534B000000435F49506A
:100590005F4741544500000010B500220268134B2C
:1005A0001A40CC680B6823434C6923438C6923436E
:1005B000CC6923430C6A23434C6A23438C6A23434C
:1005C0004C6B23438C6B23431A430260426922F035
:1005D0000702D1E90B3423431A4342610B6943609C
:1005E0004B6883608B68C36010BD00003F801CF0C7
:1005F0007047000001490860704700000C3C024051
:1006000070B504460B460026082503B909E0012B06
:1006100001D11E0205E0022B01D11E0201E04FF4C0
:10062000407600F097F80546082D28D11548006857
:1006300020F44070134908600846006830430860A1
:100640000846006820F0F80008600846006844F09A
:10065000020108430B4908600846006840F48030F6
:10066000086000F077F805460648006820F00200B0
:10067000044908600846006820F0F8000860284631
:1006800070BD0000103C024008201049096801F4C8
:100690008031B1F5803F01D1012015E00B49096897
:1006A00011F0100F01D005200EE00849096811F083
:1006B000EF0F01D0062007E00449096811F0020F8E
:1006C00001D0072000E00820704700000C3C0240E9
:1006D0000348006840F0004001490860704700008E
:1006E000103C024030B503460C46082500F032F8B5
:1006F0000546082D17D10D48006820F440700B49BD
:1007000008600846006808600846006840F001007C
:1007100008601C7000F01EF805460448006820F0D0
:10072000010002490860284630BD0000103C02402C
:100730000548006810F0004F05D0044802490C3904
:100740000860034808607047103C02402301674579
:10075000AB89EFCD00B50822FFF796FF024602E015
:10076000FFF792FF0246012AFAD0104600BD0000B2
:1007700010B50446FFF7DCFFF320FFF73BFF002036
:100780004549086080E0454800684549884207D1EE
:1007900002212020FFF734FF082801D000BFFEE728
:1007A0003E4800683F49884207D102212820FFF7D0
:1007B00027FF082801D000BFFEE7384800683A4903
:1007C000884207D102213020FFF71AFF082801D004
:1007D00000BFFEE7314800683449884207D1022152
:1007E0003820FFF70DFF082801D000BFFEE72B4897
:1007F00000682F49884207D102214020FFF700FFFF
:10080000082801D000BFFEE7244800682949884233
:1008100007D102214820FFF7F3FE082801D000BFCE
:10082000FEE71E4800682449884207D10221502073
:10083000FFF7E6FE082801D000BFFEE71748006872
:100840001749884216D3154800681C49884211D2BE
:100850001B4811490968405CFF280BD018480E4A14
:100860001268815C0D480068FFF73CFF082801D042
:1008700000BFFEE709480068401C084908600648B8
:100880000068401C0449086003480068A042FFF467
:100890007AAFFFF71DFF10BD2C0000208000002064
:1008A000000001080000020800000408000006081B
:1008B0000000080800000A0800000C0800000E08EC
:1008C000DA9E0020F0B50A4600210023002400BF74
:1008D0003DE0012505FA01F3156805EA03049C4291
:1008E00034D105684F000326BE40B5430560157935
:1008F0004E00B5400668354305601579012D02D0DC
:100900001579022D16D185684F000326BE40B543E8
:10091000856055794E00B5408668354385604568E9
:1009200001268E40B5434560456896798E40B6B243
:1009300035434560C5684F000326BE40B543C560DA
:10094000D5794E00B540C6683543C560491C1029AD
:10095000BFD3F0BDF0B5002300244D07ED0E02FA21
:1009600005F3CE1000F1200555F826504E07F70E7E
:100970000F26BE40B543CF1000F1200646F82750A1
:10098000CE1000F1200555F8265045EA0304CE109C
:1009900000F1200545F82640F0BD418370470183F2
:1009A000704730B5024612F8010BFFF72AFD0446E6
:1009B000102C01DD002030BD1078FFF722FD03462A
:1009C000102B01DD0020F6E703EB0410C0B2F2E7C4
:1009D00010B50C48006800785D2801D1002010BDDA
:1009E00008480068FFF70FFC84B200BF05480068A4
:1009F000017804480068401C024A10602C29F5D197
:100A00002046ECE78400002000BFFEE701464FF4DB
:100A100080421F4B1A800A0A1E4B1A7300BF1D4AE0
:100A2000127A12F0010FFAD01A4A127B194B19737D
:100A300000BF184A127A12F0010FFAD0154A127B41
:100A40000022144B1A7300BF124A127A12F0010FDF
:100A5000FAD0104A127B01220E4B1A7300BF0D4AC6
:100A6000127A12F0010FFAD00A4A127B0022094BC7
:100A70001A7300BF074A127A12F0010FFAD0054A22
:100A8000107B00BF4FF48042014B9B1E1A807047C1
:100A90001A0C02400030014010B501464FF480406E
:100AA000254B1880080A254B187300BF2348007A8D
:100AB00010F0010FFAD02148007B204B197300BFC2
:100AC0001E48007A10F0010FFAD01C48007B00206D
:100AD0001A4B187300BF1948007A10F0010FFAD0B2
:100AE0001648007B0220154B187300BF1348007A8C
:100AF00010F0010FFAD01148007B00200F4B187343
:100B000000BF0E48007A10F0010FFAD00B4B187B93
:100B100002020020187300BF0848007A10F0010F8D
:100B2000FAD0064B187B02434FF48043024CA41EBC
:100B30002380104610BD00001A0C02400030014016
:100B400002464FF480401F4B1880100A1E4B18734A
:100B500000BF1D48007A10F0010FFAD01A48007B40
:100B6000194B1A7300BF1848007A10F0010FFAD021
:100B70001548007B8020144B187300BF1248007A80
:100B800010F0010FFAD01048007B01200E4B1873B3
:100B900000BF0D48007A10F0010FFAD00A48007B20
:100BA0000948017300BF0848007A10F0010FFAD01D
:100BB0000548007B4FF48040024B9B1E18800120AB
:100BC000704700001A0C02400030014002464FF40A
:100BD0008040244B1880100A234B187300BF224812
:100BE000007A10F0010FFAD01F48007B1E4B1A73D9
:100BF00000BF1D48007A10F0010FFAD01A48007BA0
:100C00008020194B187300BF1748007A10F0010FAD
:100C1000FAD01548007B0220134B187300BF12480E
:100C2000007A10F0010FFAD00F48007B080A0E4B33
:100C3000187300BF0C48007A10F0010FFAD00A4870
:100C4000007B094B197300BF0748007A10F0010FB1
:100C5000FAD00548007B4FF48040024B9B1E188061
:100C6000012070471A0C0240003001401CB50446B8
:100C700001200C49087021460A48401CFFF7BAFAC7
:100C80000948C07808498978CDE9001006484378BA
:100C9000027806A10348113000F09AFC212009498E
:100CA00008601CBDDAA60020F001002049503D2557
:100CB000642E25642E25642E2564202020202020EB
:100CC00020000000740000200B48006800B9704745
:100CD0000A48008810F0800F0CD007480068C0F167
:100CE00021000749085C0549888003480068401EC8
:100CF0000149086000BFEAE77400002000100140CD
:100D0000DAA6002000BFFEE7704700000149086234
:100D10007047000000000E427047000029B1064AEB
:100D200012680243044B1A6004E0034A12688243CB
:100D3000014B1A60704700003038024029B1064A62
:100D400012680243044B1A6004E0034A12688243AB
:100D5000014B1A60704700004038024029B1064A32
:100D600012680243044B1A6004E0034A126882438B
:100D7000014B1A60704700002038024029B1064A32
:100D800012680243044B1A6004E0034A126882436B
:100D9000014B1A60704700004438024029B1064AEE
:100DA00012680243044B1A6004E0034A126882434B
:100DB000014B1A607047000024380240F0B5002152
:100DC00000220024022500260223324F3F6807F04C
:100DD0000C0121B1042905D0082937D105E02E4F97
:100DE000076036E02D4F076033E02A4F3F1F3F6812
:100DF000C7F38056274F3F1F3F6807F03F036EB190
:100E0000264FB7FBF3F7DFF88CC0ACF1040CDCF82D
:100E100000C0CCF3881C07FB0CF40CE01E4FB7FBA2
:100E2000F3F7DFF870C0ACF1040CDCF800C0CCF3D1
:100E3000881C07FB0CF4174F3F1F3F68C7F301479F
:100E40007F1C7D00B4FBF5F7076002E0124F0760DE
:100E500000BF00BF0F4F3F6807F0F0010909104FB6
:100E60007A5C0768D74047600A4F3F6807F4E05153
:100E7000890A0B4F7A5C4768D7408760054F3F6807
:100E800007F46041490B064F7A5C4768D740C7605A
:100E9000F0BD0000083802400024F40040787D01D5
:100EA0003801002021B1028842F04002028004E0B3
:100EB00002884FF6BF731A400280704710B504468F
:100EC0001148844208D101218014FFF767FF0021F7
:100ED000A014FFF763FF16E00C48844208D10121FB
:100EE0000014FFF73BFF00212014FFF737FF0AE053
:100EF0000748844207D10121C013FFF72FFF0021CB
:100F0000E013FFF72BFF10BD003001400038004018
:100F1000003C004010B50022028802F441520B88C8
:100F20004C8823438C882343CC8823430C89234358
:100F30004C8923438C892343CC8923431A43028061
:100F4000838B4FF2FF74234083830B8A038210BD8F
:100F50007047000002462A4800682A4B18604AE0A1
:100F600028480068007800B946E026480068007804
:100F7000FF2800D140E02348006800787D2800D198
:100F80003AE0204800680078222805D01D48006813
:100F9000401C1C4B18602EE01A480068401C194B7E
:100FA0001860184600680078137898421DD1002117
:100FB00008E0505C134B1B685B5C984200D004E077
:100FC000481CC1B2505C0028F3D100BF505C60B92E
:100FD0000C480068405C222807D10A480368C81CF6
:100FE0001844084B18600120704706480068401CF0
:100FF000044B186000BFB3E700BF0020F4E7000017
:10100000680000208400002010B503461D480360DE
:1010100033E01C480068007800B92FE019480068E8
:101020000078FF2800D129E01648006800787D2864
:1010300000D123E01348006800780C78A04217D153
:1010400000220DE0885C0F4C24682478A04200D078
:1010500009E00C480068401C0A4C2060501CC2B2D9
:10106000885C0028EED100BF885C08B9012010BD63
:1010700004480068401C034C2060CAE700BF002001
:10108000F5E700008400002000210020304A1268AB
:1010900042F480322E4B1A6000BF2D4A126802F4CF
:1010A0000030491C10B9B1F5C06FF6D1284A12685A
:1010B00012F4003F01D0012000E00020012845D1BA
:1010C000234A4032126842F08052214B40331A606A
:1010D000204A126842F480421E4B1A601C4A0832B1
:1010E00012681B4B08331A601A46126842F42042F9
:1010F0001A601A46126842F4A0521A60164A1B1F60
:101100001A601A1F126842F080721B1F1A6000BF1B
:101110000F4A126812F0007FFAD040F205620F4BBE
:101120001A600B4A0832126822F00302084B083397
:101130001A601A46126842F002021A6000BF044A9E
:101140000832126802F00C02082AF8D17047000039
:10115000003802400070004019544007003C024033
:1011600003200E4988804FF043600D4908608D20B0
:101170000B49543108600A493C310860081F006877
:1011800040F00100091F086005485030006840F039
:1011900001000349503108607047000000300140F1
:1011A0000864024010B51648006840F00100144978
:1011B0000860002012490831086011480068114990
:1011C00008400F4908601048091D0860081F0068A2
:1011D00020F48020091F0860002009490C310860B4
:1011E000FFF752FF4FF00060084908600748803061
:1011F000006840F4700005498031086010BD0000AF
:1012000000380240FFFFF6FE1030002408ED00E039
:1012100021B1028842F00102028004E002884FF608
:10122000FE731A400280704700220288184B9842D1
:101230000ED0184B98420BD0B0F1804F08D0164B0F
:10124000984205D0154B984202D0154B984204D1D4
:101250004FF68F731A404B881A43124B984207D0AF
:10126000114B984204D04FF6FF431A400B891A43A2
:1012700002804B68C3620B880385054B984202D0FD
:10128000044B984201D18B7A0386012383827047F5
:10129000000001400004014000040040000800403C
:1012A000000C0040001000400014004000B587B062
:1012B000072209211C48FFF74DFB07220A211A4883
:1012C000FFF748FB02208DF8080003208DF8090085
:1012D00000208DF80A0001208DF80B0040020190DB
:1012E00001A91148FFF7EEFA4FF48060019001A9BF
:1012F0000D48FFF7E7FA4FF4165003900020ADF8C1
:101300001000ADF81200ADF81400ADF818000C2074
:10131000ADF8160003A9054800F016F801210348AE
:1013200000F006F807B000BD0000024000100140C8
:1013300021B1828942F40052828104E082894DF613
:10134000FF731A40828170472DE9FF4705460E461C
:101350000024A14600BFA046B08900B100BF2C8A7E
:1013600024F44054F08804432C82AC8941F20C6090
:101370008443B08831890843718908430443AC81B0
:10138000AC8A24F44074B0890443AC826846FFF709
:1013900015FD2048854202D01F48854202D1DDF864
:1013A0000C9001E0DDF80890A88910F4004F08D0F7
:1013B00009EBC90000EB091031684900B0FBF1F7F7
:1013C00007E009EBC90000EB091031688900B0FBA8
:1013D000F1F76420B7FBF0F004012009642101FB60
:1013E0001078A88910F4004F08D0322000EBC80014
:1013F000B0FBF1F000F00700044308E0322000EBFE
:1014000008106421B0FBF1F000F00F0004432C81C0
:10141000BDE8FF87001001400014014000BFFEE757
:1014200010B5052203215F48FFF794FA0522042135
:101430005C48FFF78FFA052211465A48FFF78AFAEF
:10144000022059490871002088710220C871487132
:10145000082008605348FFF735FA202052490860F9
:101460005048FFF72FFA10204F4908604D48FFF70A
:1014700029FA4E48FFF722FD00204D490880888058
:10148000C88008814FF400704881102088810020B6
:10149000C881072008824FF4827048804348FFF7D4
:1014A00039FD01214148FFF7FDFC04203E49086059
:1014B0000120087100208871022048713D48FFF723
:1014C00001FA04213B48FFF768FA4FF440403649DF
:1014D0000860012008710020887102204871364898
:1014E000FFF7F0F94FF440413348FFF758FA012075
:1014F0002D490860087100208871022048712D482C
:10150000FFF7E0F901212B48FFF749FA4FF0C060DF
:101510002A49086025480C30486029488860002026
:10152000C8608D200861002048614FF480608861A8
:101530000020C861086248624FF4003088620020D1
:10154000C862012008630020486388631D48FFF7D4
:1015500023F84FF0C0601949086014480C30486007
:10156000194888604020C8608D20086100204861CB
:101570004FF4806088610020C861086248624FF4BF
:10158000003088620020C8620120086300204863A0
:1015900088630C481830FEF7FFFF09480B490860C4
:1015A00010BD000000040240000000200030014097
:1015B0007401002000180240000C02408801002045
:1015C0001AA7002040640240900000202001002063
:1015D0000FB4084B10B504A902AA039800F020F834
:1015E000044602A9002000F0C0F9204610BC5DF8B6
:1015F00014FB00006B1900080048704748010020E8
:1016000002E008C8121F08C1002AFAD170477047CB
:10161000002001E001C1121F002AFBD17047000029
:101620002DE9FF4F8BB005468846002667E1252847
:101630007AD100246D1CB64AA146A24601212B781E
:10164000203B01FA03F0104202D004436D1CF6E780
:1016500028782A2810D06FF02F022878A0F13001C6
:10166000092915D809EB890102EB410144F0020474
:1016700000EB01096D1CF0E758F8049BB9F1000F6D
:1016800003DA44F40054C9F1000944F002046D1C6B
:1016900028782E2817D115F8010F44F004042A28C1
:1016A0000ED06FF02F022878A0F1300109290AD856
:1016B0000AEB8A0102EB410100EB010A6D1CF2E723
:1016C00058F804AB6D1C28786C280FD006DC4C2829
:1016D00017D068280DD06A2814D104E0742810D0DF
:1016E0007A280FD10DE044F400140AE044F4801489
:1016F00001E044F440146978814202D16D1C04F584
:1017000080146D1C2878692866D007DC002876D004
:10171000632828D0642807D15EE005E06E2808D051
:1017200073282AD075287AD0DDE90D129047761CEF
:10173000E4E0C4F30250022809D003280DD0D8F801
:10174000001004280DD00E6008F10408D6E0D8F887
:101750000010F217C1E90062F6E7D8F800100E8019
:10176000F2E70E70F0E758F8041B8DF80010002027
:101770008DF80100EB46012003E058F804BB4FF060
:10178000FF3061074FF0000701D40AE07F1C574586
:101790000DDA8742FADB1BF807100029F6D106E0C4
:1017A0007F1C8742FCDB1BF807100029F8D1DDE91C
:1017B0000D23A9EB07008146214600F0BEF8304416
:1017C000C61904E0DDE90D121BF8010B90477F1EDE
:1017D000F8D2214648468CE058F8040BC4F3025175
:1017E0004FF00A0B032900D100B2042900D140B206
:1017F000002806DAC0F100004FF02D0104E082E07D
:101800000DE0210504D52B218DF82810012103E0DE
:10181000E10710D02021F7E708AF089114E058F84D
:10182000040BC4F302514FF00A0B032900D180B21C
:10183000042900D1C0B20021EEE75946FEF7F0FCC2
:1018400001F1300107F8011D0028F6D1ADEB0700CA
:1018500000F1200B600702D524F4803401E04FF042
:10186000010ADA4502DDAAEB0B0000E00020824607
:1018700000EB0B0108980144A9EB01000990E0037B
:1018800006D4DDE90D232146099800F056F80644F8
:10189000002008E00AA8DDE90D1210F809009047C1
:1018A000761C09F10100089981468842F2DBE003C9
:1018B0000CD5DDE90D232146099800F03EF80644D9
:1018C00004E0DDE90D1230209047761CBAF10001EA
:1018D000AAF1010AF5DC05E0DDE90D1217F8010BAC
:1018E0009047761CBBF10001ABF1010BF4DC0998C9
:1018F0002146DDE90D2300F00DF806446D1C287823
:1019000000287FF494AE0FB03046BDE8F08F0000A1
:10191000092801002DE9F0410446002517461E461E
:10192000880405D406E039462020B04705F10105BA
:10193000641EF8D52846BDE8F0812DE9F041044643
:10194000002590461E46C80301D5302700E0202719
:10195000880405D506E041463846B04705F1010543
:10196000641EF8D52846BDE8F0810A68531C0B6058
:101970001070704710B504464FF4804101EB04210C
:10198000491C88B20821FFF7DBF800BF4FF4804103
:1019900001EB0421491C88B2FFF738F80028F5D183
:1019A00010BD0146CA0202F5404290B2704701469E
:1019B000CA0202F5004290B270470000FE488068FB
:1019C00040F48050FC4988600121FC48FFF7A6F9EB
:1019D000012141F21000FFF7D1F90121F848FFF78A
:1019E000ADF90120FFF792F9F648006840F48070E5
:1019F000F4490860F4488068F449884246D0F448C5
:101A00000068F4490840B0F1005F3FD1F048006A37
:101A1000F1490860EE48406AF0490860EC4830300F
:101A2000EF490860EC480068B0F5503F00D92EE05F
:101A3000EA480068D0B10120EA49886000240AE041
:101A4000E74800680068E7490860E5480068001D4D
:101A5000E3490860641CE04800688442F0D3E14830
:101A60000068DE490968884200D010E0D848406824
:101A7000DD49086008460068DC490860D449086808
:101A800080F3088800BFD9480068804700BF022063
:101A9000D7490871002088710220C87148714FF43D
:101AA000E0500860D348FEF70DFF06220A21D14816
:101AB000FEF750FF06220B21CE48FEF74BFF062211
:101AC0000C21CC48FEF746FF4FF44050C84908604F
:101AD000012008710020887102204871C648FEF775
:101AE000F1FEC648FFF7EAF90020C5490880888062
:101AF000C88008814FF40070488128208881002028
:101B0000C881072008824FF482704880BB48FFF7E5
:101B100001FA0121B948FFF7C5F93220B949087027
:101B200064204870C92088709320C87026200871EE
:101B30004C204871992088713220C8716420087245
:101B4000C9204872932088722620C8724C200873DE
:101B5000992048734FF48051A748FEF71EFF4FF4B9
:101B60000051A548FEF719FFA4480C300088A6498B
:101B700008600020A1490C31088000BF9F48083050
:101B8000008810F0010FF9D09C480C3000889E4965
:101B900008604FF400519848FEF701FF002405E06B
:101BA00096480830008898490860641CB4F5FA7FAC
:101BB000F6DB4FF400519048FEF7EFFE4FF48051F2
:101BC0008D48FEF7ECFE00252BE08C480C30008899
:101BD0008D4908608B48405D88490C31088000BF02
:101BE00086480830008810F0010FF9D083480C3087
:101BF0000088854908604FF400517F48FEF7CFFE0A
:101C0000002405E07D48083000887F490860641C96
:101C1000B4F5FA7FF6DB4FF400517748FEF7BDFECE
:101C20006D1C0E2DD1DB4FF480517348FEF7B5FECD
:101C300000217248FFF736F97048FFF73FF900209E
:101C40006F4908804FF4006088800020C8800881B8
:101C50004FF400704881282088810020C881072027
:101C600008824FF4827048806448FFF753F90121DD
:101C70006248FFF717F9FEF7DFFB534880685349C6
:101C800088420CD15048C06848B14F48C0685F498D
:101C900008604D48406988604B48006948600020F2
:101CA000494988605A4858490860002418E0564855
:101CB00000680068574908600846006800B909E0F4
:101CC000544800685449884203D95048C078514963
:101CD000086007E0641C4C480068001D4A49086021
:101CE000082CE4DB00BF4D48006840084C49B0FBBD
:101CF000F1F0401E4B49088000204880401E48609B
:101D00000020088188724FF08040FFF78DFA012192
:101D10008807FFF77DFAFFF783FB01214248FEF7B2
:101D20003CFE00204FF0804148620846406A3F492F
:101D300008443549086000BF4FF08040406A32498E
:101D400009688842F8D301213748FEF728FE0020B1
:101D50004FF0804148620846406A354908442A49A4
:101D6000086000BF4FF08040406A274909688842F8
:101D7000F8D300202F4908602648006822490860EF
:101D80000846006842F21071B0FBF1F004041E48EE
:101D90000068B0FBF1F201FB12001B490860084625
:101DA00000684FF47A71B0FBF1F004EB0034164890
:101DB0000068B0FBF1F23FE0002004E07F10640017
:101DC0000180001000700040004002407155481230
:101DD000000001080000FE2F1C0000202000002051
:101DE00024000020003002408C00002088000020E9
:101DF0000000002000080240000C0240003C0040AF
:101E000074010020DA9E00202C000020F001002048
:101E10000078FF1F140000209999990024010020E8
:101E200040420F004C01002000180240A086010033
:101E300020A107007000002001FB1200FD4908608E
:101E4000084600686421B0FBF1F004EB0024F94877
:101E50000068B0FBF1F201FB1200F6490860084689
:101E600000680A21B0FBF1F004EB0014F1480068AF
:101E7000B0FBF1F201FB1200EE4908600846006871
:101E800020440860FA210920FEF75AFECE210A20DC
:101E9000FEF756FE10210B20FEF752FEE5480068C3
:101EA000C0F307410C20FEF74BFEE2480068C0F388
:101EB00007210D20FEF744FEDE480068C1B20E2067
:101EC000FEF73EFEDC4800F0A4FDDB48083000F0E1
:101ED000B3FDD948001D00F07BFD4FF47A6000F09F
:101EE00091FD032000F087FD00F0B9FD01214FF4C2
:101EF0008E40FEF725FE502144F20470FEF766FE88
:101F00004CF6CC40CD49086045F25550086004209D
:101F100048604FF47A7088604AF6AA200860002072
:101F20004FF0804148620846406AC5490844C549A7
:101F300008600020C4490860C4490860FFF7B6F98A
:101F4000C348FEF793FE27E34AF6AA20BB49086080
:101F5000FEF7BAFE4FF08040406ABA4909688842ED
:101F60007DD900204FF0804148620846406AB4495C
:101F70000844B4490860B4480068401CB24908608D
:101F80000846006840F6B83188420FD94CF6CC407C
:101F9000AA49086045F255500860012048601020A9
:101FA00088604AF6AA20086000BFFEE7A7480068DC
:101FB000401CA649086008460068032804DD00208C
:101FC00008602120A3490860A3480068401CA2497A
:101FD00008600846006810F0040F20D04FF400514C
:101FE0009E48FEF7DAFC9E4800889249086045F258
:101FF00055509B49088000BF9948001F008810F089
:10200000010FF9D0964800888A4908604FF40051C2
:102010009248FEF7C4FC00208F49086025E04FF489
:1020200000518E48FEF7B9FC8D4800888149086050
:102030008C48008820B14AF6AA208949088002E02D
:1020400000208749088000BF8548001F008810F0E5
:10205000010FF9D0824800887649086000E023E04B
:102060004FF400517D48FEF79AFC7E480088B0F599
:102070007A7F19DD7B480088401E7A49088008462F
:102080000088B0F57A7F0FDC4CF6CC406B490860D5
:1020900045F25550086001204860102088604AF6DB
:1020A000AA20086000BFFEE76F480068002871D0D2
:1020B0006D480068C01E06281FD2DFE800F0B9B8DE
:1020C0001E93B70369A16B48FEF79EFFB0B16A4843
:1020D0006AA102686748FFF77BFA6648FEF782F854
:1020E0006A49086063486A49086003205E490860DD
:1020F000002068490860684908603EE267A15D48C1
:10210000FEF782FFB8B1674B5B4867A10268594888
:10211000FFF75EFA5748FEF765F85C4908605548D6
:102120005B49086003205049086000205949086055
:102130005949086021E25FA14E48FEF765FF50B3A0
:102140005E4802684C485E4903684A48FFF740FA17
:102150004848FEF747F84D49086046494B4A12681F
:10216000881858490A6858490968FEF729F8474805
:102170000068544909680844444908603D48444996
:10218000086003203849086000204249086042493D
:102190000860F2E1F2E1FFE74CA13648FEF734FFB8
:1021A00070B1494800683A49086000203949086020
:1021B000444800683549086003202B490860DCE189
:1021C000454840683249086000203249086042486A
:1021D000C06841494968401A2C49086003202249D7
:1021E0000860CAE11F480088F8B93CA12148FEF701
:1021F0000BFF00281DD010E03B48006810F4001FC2
:1022000000D10AE04FF480401449183108800020C2
:10221000364988803649086000BF35480068012883
:10222000EAD027499031334866E0A2E0DBE098E14C
:102230006CE1CBE02C000020F001002000300040D9
:10224000A08601003000002034000020780000202B
:102250000C4500087400002038000020000C0240EB
:102260000C3C0040280000204000002053746174A2
:10227000757300009A020020140000202530366C8F
:10228000642C52756E20424F4F54210050000020A4
:10229000640000204C00002044000020566572734A
:1022A000696F6E003C2C00082530366C643B25734A
:1022B0000000000043666746696C650000000E0878
:1022C0002C4500085C00002068000020544D436F3E
:1022D0006E66696700000000FC44000872756E6D50
:1022E00061696E3D7B0000000064024000300140E7
:1022F00070000020DA9E0020FFF76AF9FE48FDF723
:1023000071FFFE49086000230846006882B2FA495E
:10231000072000F01BFB00204FF08041486200BF07
:102320004FF08040406A4CF250318842F8D3072089
:10233000FFF720FB00204FF08041486200BF4FF0C4
:102340008040406A4CF250318842F8D30020EC497A
:1023500088604CF6CC40EB49086045F25550086067
:1023600001204860102088604AF6AA20086000BF5B
:10237000FEE7E548E549086000241BE0E348006803
:102380000078212804D1E1480068401CDF4908603A
:10239000DE48006800787D2800D10EE0DB48006848
:1023A000FEF7FFFAD4490855D8480068801CD74981
:1023B0000860641CB4F5806FE0DB00BF14B12046F8
:1023C000FEF7D6F94FF47F70D1490880D149CA4849
:1023D000FFF7FEF8C848FDF705FFC849086004206C
:1023E000CD490860C9E0CA480088D0BBCBA1C64827
:1023F000FEF70AFEB0B3C548006800783A2803D05B
:102400000520C5490860B8E0C0480068401CBF49C5
:102410000860BF480088401CBD490880BB48006870
:10242000FEF7BFFA0006C0490860B8480068801C83
:10243000B649086008460068FEF7B3FABA49096869
:1024400041EA0040B8490860B0480068801CAF49C4
:102450000860B5480068B5490860B548FEF706FC55
:102460000CE007E0FFE70020A44908600520AA4926
:1024700008604AE0A448A549086000BF002416E0AF
:10248000A248006800787D2804D0A0480068007841
:10249000212800D10EE09D480068FEF782FA964997
:1024A00008559A480068801C98490860641CB4F577
:1024B000806FE5DB00BF14B12046FEF759F9934861
:1024C0000068401C9149086000209A49086001207A
:1024D00091490860002415E08C480068007828B114
:1024E0008A48006800788849085500E00CE0874871
:1024F0000068401C854908608E480068401C8D4972
:102500000860641CFA2CE7DB00BF36E08A480068EC
:10251000B0F5FA7F24D97948006808BB002414E09C
:10252000864800688649096888420CD28548006858
:1025300082490968405C7049085580480068401C21
:102540007E49086000E003E0641CB4F5967FE7DB99
:1025500000BF14B16948046002E004206E490860BD
:102560000BE075480068B0F5006F05D1634800685E
:1025700010B905206849086000BF00BF72480068B4
:1025800058B94FF4804071490880FEF7E9FD6E4864
:102590000068401C6C49086051E16B4800680128E4
:1025A0000FD16B48006810F4001F00D147E14FF4D1
:1025B00080406649891E08800020664988806249FB
:1025C000086065480068007900F02000202800D0ED
:1025D00035E16148006890F82C0014287ED05E48F0
:1025E000006890F82C00C8B1132804D0172833D005
:1025F0001C2812D125E0022144F20170FEF7A0FA56
:1026000000BF44F20170FEF701FA0028F9D14949F0
:10261000086052490860404908600EE1012144F217
:102620000170FEF78DFA00BF44F20170FEF7EEF97B
:102630000028F9D13F4908604849086036490860D8
:10264000FBE00720FFF796F900203A49086043496C
:10265000086031490860F0E03F48006890F8861053
:102660003D48006890F8850001EB00203249086081
:1026700029480068062875D2DFE800F00304DDC0B1
:10268000C1D200BF3448006890F88C10324800680E
:1026900090F88B0001EB0020314908600846006883
:1026A00040B308460068642801D9642008601648D1
:1026B000204A126881182A48006882B2072000F078
:1026C000FFF815480068B0B90F48007847284AD18C
:1026D0000D484078452846D10B4800E0AEE08078B0
:1026E000542840D10848C07820283CD108200A4905
:1026F00008604FE081E04DE0DA9E002044000020B9
:1027000000400240003000409A0200208400002077
:102710002800002010460008400000204669726D25
:102720004845583D7B0000007C00002080000020D0
:102730001E4500083C000020600000204C000020E6
:102740005000002064000020700000201A0C02409D
:1027500000640240003001402001002048000020B9
:102760001C00002067E03748007850280FD135481A
:1027700040784F280BD133488078532807D131480F
:10278000C078542803D101202F49086002E00520B9
:102790002D4908602C480068012819D1002413E055
:1027A0002A48006820442749085C212802D07D2857
:1027B00008D103E007202449086003E006202249ED
:1027C000086000BF00BF641C214800688442E7D352
:1027D0001E4800681E49096808441C490860002119
:1027E00018481A4A126881541848006849F23E4154
:1027F000884202D90520144908601CE000BF154832
:10280000006860B100231348006882B212490720B3
:1028100000F09CF80020114908600E4908600AE0A9
:102820000720FFF7A7F80020084908600C49086056
:102830000549086000BF00BF00BF00BF00BFFFF731
:1028400083BB00009A020020400000203C000020D2
:102850001C00002044000020DA9E002060000020C0
:10286000480000202DE9F0478246894616461C465E
:10287000C9F30A085046FFF794F800EB080508EB87
:102880000400B0F5006F14DDC8F500618FB23A4660
:102890003146A8B200F0FEF83E44E11B8FB250462C
:1028A000FFF77FF805463A463146284600F0F2F831
:1028B00004E022463146A8B200F0ECF8BDE8F0870B
:1028C0002DE9F04104460E4615460027002D19DD7E
:1028D0002A463146204600F018F84FF4804101EBBB
:1028E0000421491C88B24021FEF72AF900BF4FF4A9
:1028F000804101EB0421491C88B2FEF787F80028CB
:10290000F5D12F463846BDE8F081F0B504460E46B5
:1029100015464FF4804202EB0422283291B2084659
:10292000FEF7BAF807462B46324639462046FFF7EF
:1029300099FF79198FB24FF4804101EB04212831BE
:102940008AB239461046FEF741F9F0BD2DE9F04153
:1029500004460D4616461F4632462946204600F0DC
:1029600016F84FF4804101EB0421491C88B2202164
:10297000FEF7E6F800BF4FF4804101EB0421491C4B
:1029800088B2FEF743F80028F5D1BDE8F081F0B534
:1029900004460F4615464FF4804202EB04222432CF
:1029A00091B20846FEF778F806462B46324639467D
:1029B000204600F017F971198EB24FF4804101EBF7
:1029C000042124318AB231461046FEF7FFF8F0BDEB
:1029D00010B5044621780120FEF7B2F86178022094
:1029E000FEF7AEF8A1780320FEF7AAF8E1780420FC
:1029F000FEF7A6F810BD10B5044621461920FEF7D3
:102A00009FF810BD10B5044621461720FEF7DEF8EA
:102A100010BD10B5044621780F20FEF791F86178BB
:102A20001020FEF78DF8A1781120FEF789F8E178E3
:102A30001220FEF785F810BD10B504462178052058
:102A4000FEF77EF861780620FEF77AF8A178072075
:102A5000FEF776F8E1780820FEF772F810BD10B5A1
:102A6000002414E04FF4804101EB04211F318AB2AD
:102A700002211046FEF764F84FF4804101EB042177
:102A80001E318AB202211046FEF75AF8641C082C47
:102A9000E8DB10BD70B503460C4600214FF48040C2
:102AA000234D28805818000A224D287300BF214862
:102AB000007A10F0010FFAD01E48007B58181D4D07
:102AC000287300BF1B48007A10F0010FFAD0194894
:102AD000007BC2F30620174D287300BF1548007A0B
:102AE00010F0010FFAD01348007B124D2A7300BF7B
:102AF0001048007A10F0010FFAD00E48007B002138
:102B00000DE000200B4D287300BF0A48007A10F03A
:102B1000010FFAD0074D287B6054481C81B29142C6
:102B2000EFDB4FF48045024EB61E3580104670BD77
:102B30001A0C02400030014070B503460C460021DB
:102B40000AB9002070BD4FF48040244D28805818E9
:102B5000000A234D287300BF2148007A10F0010FAE
:102B6000FAD01F48007B58181D4D287300BF1C4821
:102B7000007A10F0010FFAD01948007BC2F306204A
:102B800040F08000164D287300BF1548007A10F001
:102B9000010FFAD01248007B114D2A7300BF104874
:102BA000007A10F0010FFAD00D48007B00210CE0F4
:102BB000605C0B4D287300BF0948007A10F0010FCC
:102BC000FAD00748007B481C81B29142F0DB4FF4F9
:102BD0008045024EB61E35801046B3E71A0C0240FF
:102BE000003001402DE9F0478246884691461C4658
:102BF000C9F30A075046FEF7DAFEC5193819B0F5D1
:102C0000006F14DDC7F500618EB232464146A8B2AE
:102C1000FFF792FFB044A11B8EB25046FEF7C7FEED
:102C20000546324641462846FFF786FF04E0224625
:102C30004146A8B2FFF780FFBDE8F08753494E44F4
:102C4000303A31342E30362E323031332020383A7B
:102C500034363A31302C3433003C21444F435459FC
:102C600050452068746D6C3E0D0A3C68746D6C3E76
:102C70000D0A3C686561643E0D0A3C6D6574612017
:102C8000636861727365743D225554462D38222065
:102C90002F3E0D0A3C7469746C653ED09ED0B1D055
:102CA000BDD0BED0B2D0BBD0B5D0BDD0B8D0B5208D
:102CB000D0BFD180D0BED0B3D180D0B0D0BCD0BC3A
:102CC000D18B20D0BAD0BED0BDD182D180D0BED0E1
:102CD000BBD0BBD0B5D180D0B03C2F7469746C65CB
:102CE0003E0D0A3C7374796C653E0D0A09626F648F
:102CF00079207B20666F6E742D73697A653A203176
:102D0000656D3B20666F6E742D66616D696C793AF6
:102D100020417269616C2C2048656C76657469632A
:102D2000612C2073616E732D73657269663B20633D
:102D30006F6C6F723A20233232323B206D617267C2
:102D4000696E3A2031656D3B7D0D0A096469762014
:102D50007B6D617267696E3A2032656D20303B2071
:102D60006C696E652D6865696768743A2031353025
:102D7000253B207D0D0A09696E707574207B206DDE
:102D8000617267696E3A20302032656D3B207D0D9F
:102D90000A09627574746F6E207B20646973706CAD
:102DA00061793A20626C6F636B3B20706164646987
:102DB0006E673A202E35656D2031656D3B206D6163
:102DC0007267696E3A2032656D20303B207D0D0AB6
:102DD000096831207B206D617267696E3A2030206E
:102DE000302031656D3B20666F6E742D73697A6596
:102DF0003A20323030253B20666F6E742D7765693E
:102E00006768743A206E6F726D616C3B207D0D0AAD
:102E1000092366696C652D696E666F207B20686585
:102E2000696768743A2037656D3B207D0D0A092378
:102E3000737461747573207B20636F6C6F723A20BA
:102E4000236630303B20666F6E742D73697A653A65
:102E500020313530253B20746578742D616C6967AD
:102E60006E3A2063656E7465723B207D0D0A0923FE
:102E7000696E7374616C6C207B207669736962691A
:102E80006C6974793A2068696464656E3B207D0DD5
:102E90000A3C2F7374796C653E0D0A3C2F6865619E
:102EA000643E0D0A3C626F64793E0D0A3C68313E17
:102EB000D0A0D0B5D0B6D0B8D0BC20D0BED0B1D084
:102EC000BDD0BED0B2D0BBD0B5D0BDD0B8D18F2090
:102ED000D0BFD180D0BED0B3D180D0B0D0BCD0BC18
:102EE000D18B20D0BAD0BED0BDD182D180D0BED0BF
:102EF000BBD0BBD0B5D180D0B03C2F68313E0D0ADD
:102F00003C627574746F6E20747970653D226275D1
:102F100074746F6E222069643D2265786974222082
:102F20007469746C653D22D092D18BD0B9D182D0B6
:102F3000B820D0B8D0B720D180D0B5D0B6D0B8D0D6
:102F4000BCD0B020D0BFD180D0BED0B3D180D0B063
:102F5000D0BCD0BCD0B8D180D0BED0B2D0B0D0BD63
:102F6000D0B8D18F223ED092D18BD0B9D182D0B8F7
:102F700020D0B8D0B720D180D0B5D0B6D0B8D0BC92
:102F8000D0B020D0BED0B1D0BDD0BED0B2D0BBD09A
:102F9000B5D0BDD0B8D18F20D0BFD180D0BED0B3F6
:102FA000D180D0B0D0BCD0BCD18B3C2F62757474B2
:102FB0006F6E3E0D0A3C6469763ED092D18BD0B1E3
:102FC000D0B5D180D0B8D182D0B520D184D0B0D006
:102FD000B9D0BB20D0BFD180D0BED0B3D180D0B0CB
:102FE000D0BCD0BCD18B3A3C696E707574207479BA
:102FF00070653D2266696C65222069643D226669C0
:103000006C6522206175746F636F6D706C6574659B
:103010003D226F666622202F3E3C2F6469763E0D6E
:103020000A3C6469762069643D2266696C652D6995
:103030006E666F223E3C2F6469763E0D0A3C6275D7
:1030400074746F6E20747970653D22627574746F4C
:103050006E222069643D22696E7374616C6C22205B
:103060007469746C653D22D0A3D181D182D0B0D077
:10307000BDD0BED0B2D0B8D182D18C20D0B2D18B4D
:10308000D0B1D180D0B0D0BDD0BDD183D18E20D031
:10309000BFD180D0BED0B3D180D0B0D0BCD0BCD155
:1030A00083223ED0A3D181D182D0B0D0BDD0BED0BA
:1030B000B2D0B8D182D18C20D0B2D18BD0B1D18056
:1030C000D0B0D0BDD0BDD183D18E20D0BFD180D0E3
:1030D000BED0B3D180D0B0D0BCD0BCD1833C2F62A5
:1030E0007574746F6E3E0D0A3C6469762069643DA8
:1030F00022737461747573223E3C2F6469763E0DB1
:103100000A3C7363726970743E0D0A7661722064C2
:103110003D222C222C663D22223B66756E6374692B
:103120006F6E20672862297B72657475726E20311C
:10313000303E623F2230222B623A22222B627D6691
:10314000756E6374696F6E206828297B666F7228BC
:1031500076617220623D5B66756E6374696F6E287E
:10316000297B72657475726E206E657720584D4CA0
:1031700048747470526571756573747D2C66756ED4
:103180006374696F6E28297B72657475726E206E28
:10319000657720416374697665584F626A65637428
:1031A00028224D73786D6C322E584D4C4854545033
:1031B00022297D2C66756E6374696F6E28297B7277
:1031C000657475726E206E657720416374697665EB
:1031D000584F626A65637428224D73786D6C332E84
:1031E000584D4C4854545022297D2C66756E63749A
:1031F000696F6E28297B72657475726E206E6577B3
:1032000020416374697665584F626A656374282249
:103210004D6963726F736F66742E584D4C485454E9
:103220005022297D5D2C633D21312C613D303B6175
:103230003C622E6C656E6774683B612B2B297B7436
:1032400072797B633D625B615D28297D6361746394
:10325000682872297B636F6E74696E75657D627212
:1032600065616B7D72657475726E20637D66756EC7
:103270006374696F6E206B28622C632C61297B62FA
:103280002E6164644576656E744C697374656E6511
:10329000723F622E6164644576656E744C69737426
:1032A000656E657228632C612C2131293A622E618A
:1032B00074746163684576656E743F622E617474E0
:1032C0006163684576656E7428226F6E222B632CCD
:1032D00061293A625B226F6E222B635D3D617D0A3C
:1032E00066756E6374696F6E206C28622C63297B2F
:1032F00076617220613D622B322A633B613D642E10
:103300006368617241742861292B642E636861725D
:10331000417428612B31293B32213D612E6C656E51
:103320006774683F613D6E756C6C3A28613D7061F1
:10333000727365496E7428612C3136292C613D69A0
:10334000734E614E2861293F6E756C6C3A61293B62
:1033500072657475726E20537472696E672E667230
:103360006F6D43686172436F64652861297D66757E
:103370006E6374696F6E206D28622C63297B7661A1
:103380007220633D632B31322C613D7B7479706513
:103390003A622C643A7061727365496E74286C28C5
:1033A000632C30292B6C28632C31292C3130292CAB
:1033B0006D3A7061727365496E74286C28632C33A2
:1033C000292B6C28632C34292C3130292C793A7024
:1033D00061727365496E74286C28632C36292B6CD6
:1033E00028632C37292B6C28632C38292B6C2863F5
:1033F0002C39292C3130292C683A70617273654957
:103400006E74286C28632C3131292B6C28632C3185
:1034100032292C3130292C693A7061727365496EFA
:1034200074286C28632C3134292B6C28632C31359B
:10343000292C3130297D3B72657475726E20612EA6
:10344000747970652B223A222B6728612E64292B10
:10345000222E222B6728612E6D292B222E222B67EC
:1034600028612E79292B2220222B6728612E68299A
:103470002B223A222B6728612E69297D66756E639F
:1034800074696F6E206E2862297B646F63756D6549
:103490006E742E676574456C656D656E744279490E
:1034A00064282266696C652D696E666F22292E6913
:1034B0006E6E657248544D4C3D627D0A66756E6352
:1034C00074696F6E206F2862297B646F63756D6508
:1034D0006E742E676574456C656D656E74427949CE
:1034E00064282273746174757322292E696E6E6567
:1034F0007248544D4C3D622E7265706C6163652854
:103500002F5C6E2F69672C223C6272202F3E22298D
:103510007D0A66756E6374696F6E20702862297B00
:1035200076617220633D6828293B632E6F6E726559
:1035300061647973746174656368616E67653D6623
:10354000756E6374696F6E28297B343D3D632E72FE
:10355000656164795374617465262628636C6561BE
:103560007254696D656F75742861292C6F28225C0F
:1035700075303431345C75303433355C7530343308
:10358000395C75303434315C75303434325C7530CC
:103590003433325C75303433385C75303433352035
:1035A0005C75303433325C75303434625C75303481
:1035B00033665C75303433655C75303433625C750A
:1035C000303433645C75303433355C753034336497
:1035D0005C75303433655C6E5C75303431345C75E9
:1035E000303433305C75303433645C75303433647C
:1035F0005C75303433305C7530343466205C753043
:103600003434315C75303434325C75303434305C91
:1036100075303433305C75303433645C753034333A
:10362000385C75303434365C7530343330205C753A
:10363000303433655C75303433315C753034336429
:103640005C75303433655C75303433325C753034DE
:1036500033385C75303434325C75303434315C75F9
:1036600030343466205C75303434375C7530343334
:10367000355C75303434305C75303433355C7530DE
:103680003433372035205C75303434315C75303458
:1036900033355C75303433615C75303434335C758C
:1036A000303433645C753034333422292C736574C0
:1036B00054696D656F75742866756E6374696F6E95
:1036C00028297B77696E646F772E6C6F63617469EC
:1036D0006F6E2E72656C6F616428297D2C354533C1
:1036E00029297D3B632E6F70656E2822706F73747D
:1036F000222C222F222C2130293B632E73657452F9
:103700006571756573744865616465722822436FDD
:103710006E74656E742D54797065222C0A22617066
:10372000706C69636174696F6E2F782D7777772D70
:10373000666F726D2D75726C656E636F6465642261
:10374000293B632E73656E642862293B6F28225CD7
:1037500075303431325C75303434625C75303433FA
:10376000665C75303433655C75303433625C75305B
:103770003433645C75303434665C75303433355CB6
:1037800075303434325C75303434315C75303434F7
:1037900066205C75303433345C75303433355C7599
:1037A000303433395C75303434315C753034343214
:1037B0005C75303433325C75303433385C7530349A
:1037C00033352C205C75303433665C7530343365AA
:1037D0005C75303433365C75303433305C7530347E
:1037E00033625C75303434335C75303433395C7536
:1037F000303434315C75303434325C7530343330CD
:103800002C205C75303433365C75303433345C7561
:10381000303433385C75303434325C7530343335A1
:103820002E2E2E22293B76617220613D73657454E1
:10383000696D656F75742866756E6374696F6E283F
:10384000297B632E61626F727428293B6F28225C8A
:1038500075303431615C75303433655C75303433C8
:10386000645C75303434325C75303434305C7530BF
:103870003433655C75303433625C75303433625C8C
:1038800075303433355C7530343430205C75303409
:1038900033645C7530343335205C75303433655CAB
:1038A00075303434325C75303433325C75303433D7
:1038B000355C75303434375C75303433305C75309A
:1038C0003433355C753034343222297D2C33453421
:1038D000297D0A6966282177696E646F772E4669AB
:1038E0006C657C7C2177696E646F772E46696C65A8
:1038F0005265616465727C7C2177696E646F772E96
:1039000046696C654C697374296F28225C75303484
:1039100031325C75303433305C7530343438205C8F
:1039200075303433315C75303434305C7530343359
:10393000305C75303434335C75303433375C75301B
:103940003433355C7530343430205C753034336456
:103950005C7530343335205C75303433665C7530DB
:103960003433655C75303433345C75303433345CF7
:1039700075303433355C75303434305C7530343305
:10398000365C75303433385C75303433325C7530C6
:103990003433305C75303433355C75303434322038
:1039A0005C75303433635C75303433355C7530347A
:1039B00034355C75303433305C75303433645C7569
:1039C000303433385C75303433375C7530343363BE
:1039D000205C75303433665C75303433355C75305B
:1039E0003434305C75303433355C75303433665C78
:1039F00075303434305C75303433655C7530343355
:103A0000335C75303434305C75303433305C753051
:103A10003433635C75303433635C75303433385C15
:103A200075303434305C75303433655C7530343324
:103A3000325C75303433305C75303433645C7530EF
:103A40003433385C7530343466205C75303433611F
:103A50005C75303433655C75303433645C75303498
:103A600034325C75303434305C75303433655C75B9
:103A7000303433625C75303433625C7530343335E6
:103A80005C75303434305C75303433302E5C6E5CB1
:103A90006E5C75303431325C75303433655C753052
:103AA0003434315C75303433665C75303433655C86
:103AB00075303433625C75303434635C7530343364
:103AC000375C75303434335C75303433395C753081
:103AD0003434325C75303433355C75303434315CB9
:103AE0007530343463205C75303433655C75303444
:103AF00033345C75303433645C75303433385C7522
:103B000030343363205C75303433385C7530343393
:103B100037205C75303434315C75303433625C7519
:103B2000303433355C75303433345C753034343391
:103B30005C75303434655C75303434395C753034E0
:103B400033385C7530343435205C75303433315C57
:103B500075303434305C75303433305C7530343427
:103B6000335C75303433375C75303433355C7530E5
:103B70003434305C75303433655C75303433323A0C
:103B80005C6E496E7465726E6574204578706C6FFA
:103B90007265722031302E302B2C5C6E4D6F7A693D
:103BA0006C6C612046697265666F7820332E362B07
:103BB0002C5C6E476F6F676C65204368726F6D6534
:103BC00020372E302B2C5C6E4F70657261203131A6
:103BD0002E35302B2E22292C646F63756D656E7423
:103BE0002E676574456C656D656E7442794964280D
:103BF0002266696C6522292E64697361626C656452
:103C00003D0A21303B0A6B28646F63756D656E74E5
:103C10002E676574456C656D656E744279496428DC
:103C20002266696C6522292C226368616E676522B1
:103C30002C66756E6374696F6E28297B76617220BD
:103C4000623D646F63756D656E742E676574456C57
:103C5000656D656E7442794964282266696C6522D7
:103C6000292E66696C65735B305D3B696628622945
:103C70007B76617220633D275C75303431325C7530
:103C8000303434625C75303433315C753034343008
:103C90005C75303433305C7530343364205C75309F
:103CA0003434345C75303433305C75303433395CE3
:103CB0007530343362203C656D3E22272B622E6EB8
:103CC000616D652B27223C2F656D3E2C20272B280C
:103CD000622E73697A652F31303234292E746F4623
:103CE0006978656428292B22205C75303433615C47
:103CF00075303433312E222C613D6E657720466954
:103D00006C655265616465723B612E7265616441E8
:103D100073546578742862293B612E6F6E6C6F61F5
:103D2000643D66756E6374696F6E2861297B666F8A
:103D3000722876617220613D612E746172676574CC
:103D40002E726573756C742E73706C697428223AC8
:103D5000303230303030303422292C623D5B5D2CE3
:103D6000713D312C693B693D615B712B2B5D3B29BA
:103D70007B766172206A3D692E7375627374726915
:103D80006E6728302C34292C653D7061727365494B
:103D90006E74286A2C3130293B6966282128383016
:103DA000303E657C7C3930303C6529297B693D6932
:103DB0002E73706C697428225C6E22293B303D3D65
:103DC000622E6C656E6774682626622E7075736845
:103DD00028223A222B6A293B666F72286A3D323BC1
:103DE000653D695B6A2B2B5D3B29653D652E736CD8
:103DF00069636528392C2D33292C622E7075736800
:103E00002865292C0A303D3D286A26372926266256
:103E10002E7075736828222122297D7D663D622ED1
:103E20006A6F696E282222293B643D662E73706C8E
:103E3000697428222122292E6A6F696E282222297C
:103E40003B613D642E696E6465784F662822353388
:103E50003439344534343330334122293B623D64B4
:103E60002E696E6465784F662822353334393445BF
:103E700034343537334122293B303E617C7C303E3F
:103E8000623F286E28632B223C6272202F3E3C73D7
:103E900074726F6E673E5C75303431645C753034BB
:103EA00033355C75303433615C75303433655C7543
:103EB000303434305C75303434305C753034333504
:103EC0005C75303433615C75303434325C75303459
:103ED00033645C75303434625C7530343339205C63
:103EE00075303434345C75303433305C7530343391
:103EF000395C7530343362205C75303433665C7500
:103F0000303434305C75303433655C753034333381
:103F10005C75303434305C75303433305C7530343B
:103F200033635C75303433635C7530343462213C08
:103F30002F7374726F6E673E22292C646F63756DE8
:103F4000656E742E676574456C656D656E74427937
:103F500049642822696E7374616C6C22292E737413
:103F6000796C652E7669736962696C6974793D2232
:103F700068696464656E22293A286E28632B223CA6
:103F80006272202F3E5C75303431615C75303433A1
:103F9000655C75303434305C75303434305C753089
:103FA0003433355C75303433615C75303434325CB5
:103FB00075303433645C75303434625C753034335E
:103FC00039205C75303434345C75303433305C7592
:103FD000303433395C7530343362205C75303433BF
:103FE000665C75303434305C75303433655C753004
:103FF0003433335C75303434305C75303433305C9A
:1040000075303433635C75303433635C753034340D
:1040100062213C6272202F3E3C6272202F3E5C7512
:10402000303431325C75303433355C753034343093
:104030005C75303434315C75303433385C75303411
:104040003466205C75303433665C75303434305CF3
:1040500075303433655C75303433335C75303434EB
:10406000305C75303433305C75303433635C7530BC
:104070003433635C7530343462205C7530343361C2
:104080005C75303433655C75303433645C75303462
:1040900034325C75303434305C75303433655C7583
:1040A000303433625C75303433625C7530343335B0
:1040B0005C75303434305C75303433303A203C73C6
:1040C00074726F6E673E222B0A6D282253494E3060
:1040D000222C61292B223C2F7374726F6E673E2C49
:1040E0003C6272202F3E5C75303431325C75303466
:1040F00033355C75303434305C75303434315C7554
:10410000303433385C7530343466205C7530343389
:10411000665C75303434305C75303433655C7530D2
:104120003433335C75303434305C75303433305C68
:1041300075303433635C75303433635C75303434DC
:1041400062205C75303433615C75303433655C7586
:10415000303433645C75303434345C753034333827
:104160005C75303433335C75303434335C753034E3
:1041700034305C75303433305C75303434325C75D7
:10418000303433655C75303434305C753034333002
:104190003A203C7374726F6E673E222B6D28225357
:1041A000494E57222C62292B223C2F7374726F6E5A
:1041B000673E2E22292C646F63756D656E742E67C1
:1041C0006574456C656D656E744279496428226931
:1041D0006E7374616C6C22292E7374796C652E7603
:1041E00069736962696C6974793D22766973696281
:1041F0006C6522297D7D656C7365206E28222229DD
:104200007D293B0A6B28646F63756D656E742E673C
:104210006574456C656D656E7442794964282269E0
:104220006E7374616C6C22292C22636C69636B223F
:104230002C66756E6374696F6E28297B21646F63C9
:10424000756D656E742E676574456C656D656E740D
:1042500042794964282266696C6522292E66696C58
:1042600065735B305D7C7C21663F6F28225C753016
:104270003432335C75303433615C75303433305CE8
:1042800075303433365C75303433385C75303434E3
:10429000325C7530343335205C75303433615C7595
:1042A000303433655C75303434305C7530343430E0
:1042B0005C75303433355C75303433615C75303463
:1042C00034325C75303433645C75303434625C7520
:1042D00030343339205C75303434345C75303433E9
:1042E000305C75303433395C7530343362205C7542
:1042F000303433665C75303434305C75303433655B
:104300005C75303433335C75303434305C75303444
:1043100033305C75303433635C75303433635C75D3
:104320003034346222293A7028224669726D484539
:10433000583D7B222B662B227D22297D293B0A6B4F
:1043400028646F63756D656E742E676574456C6562
:104350006D656E74427949642822657869742229F2
:104360002C22636C69636B222C66756E6374696FB3
:104370006E28297B636F6E6669726D28225C7530CA
:104380003431665C75303433655C75303433345C9D
:1043900075303434325C75303433325C75303433DC
:1043A000355C75303434305C75303433345C7530A2
:1043B0003433385C75303434325C75303433352006
:1043C0005C75303433325C75303434625C75303453
:1043D00034355C75303433655C7530343334205C8F
:1043E00075303433385C7530343337205C75303495
:1043F00034305C75303433355C75303433365C754D
:10440000303433385C75303433635C75303433307A
:10441000205C75303433655C75303433315C753015
:104420003433645C75303433655C75303433325CFE
:1044300075303433625C75303433355C7530343309
:10444000645C75303433385C7530343466205C75A8
:10445000303433665C75303434305C7530343365F9
:104460005C75303433335C75303434305C753034E3
:1044700033305C75303433635C75303433635C7572
:1044800030343462205C75303433615C75303433E1
:10449000655C75303433645C75303434325C75304F
:1044A0003434305C75303433655C75303433625C81
:1044B00075303433625C75303433355C7530343488
:1044C000305C7530343330222926267028227275EC
:1044D0006E6D61696E3D7B317D22297D293B0A3CF1
:1044E0002F7363726970743E0D0A3C2F626F64799A
:1044F0003E0D0A3C2F68746D6C3E0000648A17887C
:10450000592C000800000000FA4400085761697443
:10451000696E670046696C65206C6F616400466C6B
:104520006173682057524954452100004854545043
:104530002F312E3120323030204F4B0D0A436F6E19
:1045400074656E742D4C656E6774683A20256C64D2
:104550000D0A436F6E74656E742D547970653A2040
:104560006170706C69636174696F6E2F6F637465DD
:10457000742D73747265616D0D0A436F6E74656E90
:10458000742D446973706F736974696F6E3A20613A
:1045900074746163686D656E743B2066696C656EEA
:1045A000616D653D53696E636F6D445F2530366C98
:1045B000642E7478740D0A0D0A000000485454509B
:1045C0002F312E3120323030204F4B200D0A436FD7
:1045D0006E6E656374696F6E3A20636C6F73650D00
:1045E0000A4163636573732D436F6E74726F6C2D34
:1045F000416C6C6F772D4F726967696E3A2A0D0AAC
:104600000D0A205265616479210D0A0D0A0000002F
:10461000485454502F312E3120323030204F4B200F
:104620000D0A436F6E6E656374696F6E3A20636C3A
:104630006F73650D0A4163636573732D436F6E7409
:10464000726F6C2D416C6C6F772D4F726967696E5C
:104650003A2A0D0A0D0A00004040404040404040C8
:104660004041414141414040404040404040404045
:104670004040404040404040050202020202020227
:10468000020202020202020220202020202020201A
:10469000202002020202020202909090909090105C
:1046A000101010101010101010101010101010100A
:1046B0001010100202020202028888888888880886
:1046C000080808080808080808080808080808086A
:1046D000080808020202024058460008FC4600088A
:1046E000000000204C010000A20300084847000819
:1046F0004C0100205CAA0000101600080191123540
:1047000012011B4003052A41052A42052A43052AB6
:1047100044052A45052A46052A47051340208208F4
:104720009A410C9A420C9A430C9A440C9A450C9A62
:10473000460C9A470C81847A030A68090102030433
:08474000060708090CA910008E
:020000044002B8
:1040000001FF01FF01FF01FF01FF01FF01FF01FFB0
:0840100001FF01FF012A00007D
:040000050800018965
:00000001FF
